:020000020000FC
:1000000000C001E302BB00E007BB00E001BB02E06F
:100010000EBF0FE50DBF00E805BF09E109B9539A0E
:10002000549AECD7809902C0A7D6AED7E6D72FD284
:100030006FEFB5D14CD0FBCFE395C895319600203A
:1000400009F0089550E0BFC1F9E0E6E4F6DF0916D3
:1000500079F4F3DF081669F4F0DF071659F43196E6
:10006000C895002D3196C895F02DE02F099508957B
:10007000319631963396EACF90EF80EF21E00881F8
:1000800066D1513011F41AD0F7CF702F17D00D3040
:1000900091F0952E08815BD10D3069F0951639F4F9
:1000A000982F872F702F0AD02395233099F7088136
:1000B0004ED1951609F0089501D0F9CFD81529F43D
:1000C000C71519F454E07FC1089521970895D0E031
:1000D000C8EC0AE8702E00E0802E088138D152303A
:1000E00009F476C0D4D1A16001C0AE7F3DB73830ED
:1000F00010F458E068C1C0DF7D30B9F0092D02303E
:1001000031F49F708F707F7024D220D0EFCF9F7515
:100110008F757F75213029F4092D033011F407D034
:10012000E5CF92DF7D3009F00895A1600895715404
:100130007A3112F055E047C17059A0FF11F406D092
:100140000895F0E0E72F708101D00895F1E0E62FE7
:1001500070836A95633F10F456E035C10895639546
:10016000603012F057E02FC1F1E0E62F7081089562
:100170005BE029C1D0E0C8ECFF24EE247727BF7DE7
:100180000881CA95E3940D3041F0E1D0523039F046
:10019000B0625130A9F3F394F3CF0F2D0895B5FF5A
:1001A0007395EECF54E00FC152E00DC19F708F7078
:1001B0007F70CFD10895D0E0C8ECE93CA9F3088165
:1001C0000083319721970D30C1F75E2E6F2E089571
:1001D000D1DF743068F6062D0F3721F4052D033F6B
:1001E00009F452C0D0E0C8EC772788279927C715B3
:1001F000CAF20881ACD0523029F4982F872F702F83
:100200002197F5CFD3DFA72EF62DE52DB77FBF7E43
:10021000992788277727BB243196FF3711F4E43FCD
:1002200059F0008194D0543039F0523089F7B394AA
:10023000782F892F902FF0CF0B2D033029F0B39416
:10024000782F892F90E0F8CFB4FD02C0B061E0CFE5
:10025000ADDFA71691F118F4B860DF2ECE2EFF3770
:1002600021F4E43F11F4B3FF0FC0B3FF08C07A15C7
:1002700008F442C0FF3719F4E43F09F43DC0FF37EA
:1002800039F6E43F29F6089575DF003009F4089542
:10029000D0E0C8ECF62DE52DF33019F4E93C09F473
:1002A00009C008810083319721970D30A9F75E2E90
:1002B0006F2E089502E0502F86C03197DF2FCE2F8A
:1002C000D33019F4C93C09F46DCF088121970D3062
:1002D000B9F70E2F0C1B500E08F46394D33011F4B1
:1002E000C93C29F00881008321973197F7CF42DF7D
:1002F000003009F06DCF08953DDF003039F1062D53
:10030000033021F4052D095C0E15A0F2F62DE52D24
:10031000DF2FCE2FCE19D0400C2F502E0D2F602E58
:10032000FD1519F4EC1509F405C000810883219628
:100330003196F6CFD0E0C8ECFD2DEC2D3197088139
:1003400000830D3019F031972197F9CF0895552783
:10035000102F1D3009F416C01F75103009F402C0AB
:100360001C3011F451E0089510310AF408951B3542
:100370000AF00895103412F053E008951A310AF487
:1003800052E0089554E00895C83C19F427E075D070
:100390000AC0212F81D0C3951DE0188304C02EE32D
:1003A0006CD0D0E0C8EC7DD0183071F318831D30CC
:1003B00049F0CB3819F427E060D0F5CFCA95212F4A
:1003C0006BD0F1CF089563D0503021F4F6E0E0E730
:1003D0006CD042C0513021F4F6E0E8E966D03CC070
:1003E000523021F4F6E0E6ED60D036C0533021F40F
:1003F000F6E0E8EF5AD030C0543021F4F7E0EAE3F9
:1004000054D02AC0553021F4F7E0ECE64ED024C099
:10041000563021F4F7E0E0EA48D01EC0573021F40E
:10042000F7E0E2EE42D018C0583021F4F8E0E2E400
:100430003CD012C0593021F4F8E0E2EA36D00CC0CA
:100440005A3021F4F8E0EAED30D006C05B3021F4F8
:10045000F9E0E2E12AD000C00FE502E00EBF0FE5AF
:100460000DBF6FEFA0E0B0E012D0E1CD57D0242F48
:1004700004D0232F02D00895202F5D9BFECF59D6A4
:10048000B6FF03C05F9BFECFBF7B2CB908952DE064
:10049000F4DF2AE0F2DF08952D3011F4F8DF08953B
:1004A000ECCF5F9BFECF1CB10895C895002021F0D2
:1004B000202DE3DF3196F9CF0895F7DFE8DF0895C7
:1004C0004EDE07E007174AF001E0703019F0000F28
:1004D0007A95FBCF702F3ADE08955AE074DF9030A2
:1004E00039F0905D292FC9DF803011F420E3C5DF9A
:1004F000803019F0805D282FC0DF705D272FBDDFB1
:10050000089599278827745610F09395FCCF7C594D
:100510007A5010F08395FCCF765F0895432F46956F
:10052000469546954695405D4A3308F0495F3F70D1
:10053000305D3A3308F0395F089546FD475F4F70EC
:1005400036FD375F3F70440F440F440F440F342B88
:1005500008959330B2F4923032F0863092F48530C0
:1005600012F0763072F4882321F00AE0700F8A9539
:1005700081F7992309F4089504E68894700F9A95F9
:10058000C0F751E020CF83DF82DFF5E0E2E995DFBD
:1005900008952020202020204154544F42415349A7
:1005A000432076657273696F6E2038353135585245
:1005B0002D303331303133412E204E6F7420666F31
:1005C0007220636F6D6D65726369616C2075736510
:1005D0002E200A0D202020202020436F7079726980
:1005E00067687420323030322C2032303033206251
:1005F0007920526963686172642043617070656C30
:100600007320616C6C207269676874732072657303
:1006100065727665642E0A0D2020202020206874E3
:1006200074703A2F2F70726F6A656374732E6361F2
:100630007070656C732E6F72672020202020202040
:1006400070726F6A656374734063617070656C7318
:100650002E6F72670A0D000046726565202070617A
:100660006765733A0000202063686172733A000086
:100670004572726F7220303A20556E6B6E6F776ED6
:1006800020636F6D6D616E64206F72206F70657294
:1006900061746F722E2000004572726F7220313AC1
:1006A00020456E636F756E74657265642061207697
:1006B000616C75652074686174206973206E6F7455
:1006C000206265747765656E203020616E6420322B
:1006D00035352E2000004572726F7220323A20505C
:1006E000726F6772616D206D656D6F7279206973CD
:1006F0002066756C6C2E00004572726F7220333A62
:1007000020456E636F756E74657265642061206349
:1007100068617261637465722074686174206973C2
:10072000206E6F742061207265636F676E697A65F1
:100730006420747970652E2000004572726F7220FB
:10074000343A28696E7465726E616C206572726FDE
:1007500072202D627566666572206C696D69742001
:100760006578636565646564292000004572726F71
:100770007220353A20496E617070726F70726961D3
:100780007465207661726961626C65206E616D6569
:1007900020656E636F756E74657265642E2000004F
:1007A0004572726F7220363A20446174612073740E
:1007B00061636B2070757368206572726F72202D93
:1007C000746F6F206D616E7920617267756D656EF3
:1007D0007473206F6E206F6E65206C696E652E20BD
:1007E00000004572726F7220373A204461746120B4
:1007F000737461636B20706F70206572726F722EFC
:100800000A0D20202020202020202046756E6374B1
:10081000696F6E20747269656420746F20757365EA
:1008200020612076616C7565207468617420776141
:1008300073206E6F7420617661696C61626C652EE5
:1008400000004572726F7220383A204D616368690A
:100850006E6520737461636B206572726F720A0D2E
:1008600020202020202020202046756E6374696F90
:100870006E7320616E642F6F722063616C6C7320E5
:100880006E657374656420746F6F20646565706C49
:1008900079206F7220746F6F20636F6D706C657854
:1008A00000004572726F7220393A20474F544F2032
:1008B0006F7220474F5355422064657374696E61AF
:1008C00074696F6E206C696E6520776173206E6F3E
:1008D0007420666F756E642E00004572726F722010
:1008E000413A205370656369666965642062697482
:1008F00020706F736974696F6E2072616E67652016
:100900006F6620302E2E37206578636565646564D8
:1009100000004572726F7220423A204C696E652069
:100920006E756D62657220686173206D6F726520EF
:100930007468616E207468726565206E756D65728D
:10094000616C732000004C495320880553495A209C
:1009500094054E455720FD0750500B20FB05505085
:100960000D2002065052494EA80550525820AF059E
:1009700050524220E10650574D383106505745201D
:100980003B0650574F204706454D4954D406501A50
:100990001D20B70550501D20C005464F52205E0651
:1009A0004E455854D105501C1E20DA0550501E20CB
:1009B0004A0650501C202B065049462054065054DD
:1009C0004F20600650500420640652554E20C40744
:1009D000454E44206206414E442009064C535220A5
:1009E00010064C534C201506504F52201A06584FF3
:1009F0005220210644554D501008474F544F96063B
:100A0000474F53559A06524554559D065448454EF6
:100A10005A064B455920D90641434F20E60553411C
:100A20005645A3064C4F4144BC065045454BEC058A
:100A3000504F4B45F3054F444120A1074F444220FE
:100A4000A5074F444320A9074F444420AD074F500A
:100A5000412091074F50422095074F50432099075E
:100A60004F5044209D07494E4120B107494E422036
:100A7000B407494E4320B807494E4420BB075342B0
:100A80004120ED0643424120F40653424220FC0639
:100A9000434242200307534243200B074342432073
:100AA0001207534244201A0743424420210753446B
:100AB000412029074344412030075344422038074E
:100AC000434442203F0753444320470743444320C5
:100AD0004E07534444205607434444205D0749428F
:100AE00041206507494242207007494243207B0765
:100AF00049424420860744454C412D084453524501
:100B00004E084453434F48084453444542080000AC
:100B1000BEDCFFE7E3EFF61511F4E51521F02081C7
:100B2000BBDC3197F8CFB3DCB2DCF6E0E8E5BDDC46
:100B3000752D962D795C934009DB792FE2DCCFDCB3
:100B4000F6E0E6E6B2DC0BDBDCDCC9DCA0DC089519
:100B5000AE7FCCDA04DBD5DCC2DC99DC0895C5DAE3
:100B600024E28BDCFCDA372F81DC91DC0895AE7F48
:100B7000BDDAF5DA072FF3DAF0E0E72F0083089506
:100B8000A2FF40C0AE7FB2DAEADAA72EE8DA872FFA
:100B9000E6DAB72EF0E0E72F8083A062A860AA7F94
:100BA0000895F0E0EB2D00810A1519F003950083FC
:100BB000A06108959ADAD3DA072FD1DA701719F005
:100BC0007727C4DA08957FEFC1DA08958EDA70E0EE
:100BD000459B71E0BBDA089588DAC1DAE72FF0E0CF
:100BE0007081B4DA089581DABADA072FB8DAF0E062
:100BF000E02F7083089579DAB2DA072FB0DA700F38
:100C0000A5DA089572DAABDA072FA9DA701B9EDA3B
:100C100008956BDAA4DA072FA2DA702397DA089521
:100C200064DA9DDA769592DA08955FDA98DA770FCA
:100C30008DDA08955ADA93DA072F91DA702B86DA73
:100C4000089553DA8CDA072F8ADA70277FDA08954D
:100C500071E07CDA089549DA82DA072F80DA7017BA
:100C60001EC043DA01E80FBD0EBD8D9A78DA00E0B0
:100C70000BBD7ABD089539DA03E80FBD01E00EBD62
:100C8000BD9A6DDA072F6BDA7BBD0ABD089500E0CF
:100C90000FBD08952ADA63DA072F61DA071770E0CB
:100CA000BAF6B1F253DA089520DA59DA772309F067
:100CB000A26008950DB70E5F0DBF0895A46008955A
:100CC00014DA0895B26008954881F8D9388135DC86
:100CD000732F3CDAF3D909DA089507DA40DA472F9F
:100CE000FFE7E3EF0AC0F61511F45E16E8F40081A1
:100CF0000D3011F03197F7CF319777278827992753
:100D0000F61511F45E1680F4008121DB523029F4CF
:100D1000982F872F702F3197F3CF9F708F707F7030
:100D200018DC471701F7089559E04DCBD6DFDF2FC8
:100D3000CE2F0895D2DFA06C0895B2FF02C0B1603B
:100D40000895B26008956FEF752D00DA762DFED903
:100D5000DFE7CFEFEFEFF1E00881E199FECFFFBBD6
:100D6000EEBB0DBBE29AE19AD33011F4C93C19F005
:100D700031972197F1CF0895DFE7CFEFEFEFF1E063
:100D8000E199FECFFFBBEEBBE09A0DB30883D330F1
:100D900011F4C93C19F031972197F2CF6DEFDFD9EB
:100DA000672EDDD9572E0895A0D9D9D9272F65DB15
:100DB00008955F9BFECF7CB1733009F4B260C6D951
:100DC000089593D9CCD908E020E3771F08F421E3F4
:100DD00054DB0A95C9F75BDB089587D971DBBFD96E
:100DE0000BB3072B02BB089580D96ADBB8D9709585
:100DF0000BB3072302BB089578D962DBB0D908B3DF
:100E0000072B02BB089571D95BDBA9D9709508B394
:100E1000072302BB089569D953DBA1D905B3072B7A
:100E200002BB089562D94CDB9AD9709505B30723AC
:100E300002BB08955AD944DB92D902B3072B02BBF7
:100E4000089553D93DDB8BD9709502B3072302BBBC
:100E500008954BD935DB83D90AB3072B0ABB089514
:100E600044D92EDB7CD970950AB307230ABB0895B9
:100E70003CD926DB74D907B3072B07BB089535D9B6
:100E80001FDB6DD9709507B3072307BB08952DD9D4
:100E900017DB65D904B3072B04BB089526D910DBF3
:100EA0005ED9709504B3072304BB08951ED908DBEF
:100EB00056D901B3072B01BB089517D901DB4FD9D0
:100EC000709501B307230ABB08950FD9F9DA47D902
:100ED00009B3072370E0002309F471E037D90895BE
:100EE00004D9EEDA3CD906B3072370E0002309F4F5
:100EF00071E02CD90895F9D8E3DA31D903B3072387
:100F000070E0002309F471E021D90895EED8D8DA11
:100F100026D900B3072370E0002309F471E016D945
:100F20000895E3D81CD97BBB0895DFD818D978BBC6
:100F30000895DBD814D975BB0895D7D810D972BBE2
:100F40000895D3D80CD97ABB0895CFD808D977BBE8
:100F50000895CBD804D974BB0895C7D800D971BB04
:100F6000089579B3F3D8089576B37C7FEFD80895C8
:100F700073B3ECD8089570B37C7FE8D808954272BB
:100F800065616B200A0D0000DFE7C3EF6FEFA16022
:100F9000D0D0A5FF03C0CC2EDD2EAF7DA4FF03C0B3
:100FA000DD2DCC2DAF7EA6FF03C0EC2EFD2EAF7B3A
:100FB000A7FF04C0DF2FCE2FB460AF77B0FF03C010
:100FC000DF2DCE2DBA7FB1FF04C043D0D62DC52D65
:100FD000BD7FD61511F45C1678F40881B8D9A1FF4D
:100FE00004C0543011F02197D1CFAD7F523011F4AD
:100FF0002197CCCF7BD8CACF0895C5DA0FE7602EF2
:1010000003EF502EF62DE52D6FEFA0E0B0E000E0ED
:10101000F33011F4E93C19F000833197F9CF0895CA
:10102000FFE7E3EFF33011F4E93C41F030811EDAE1
:1010300020E223DA20E221DA3197F4CF28DA27DA26
:10104000362D14DA20E219DA352D10DA20DA1FDA1B
:101050000895FFE0EEE729DA089547D880D8992768
:10106000882755270027772361F09A958A955A9506
:101070004A95F1F70A95E1F7D1F7C1F7B1F77A95FB
:10108000F2CF089532D86BD8172F88940BD00895DB
:101090002CD865D8172F089405D0089527D0712F24
:1010A00055D8089501B3077E01BB02B3086102BBA6
:1010B00099E0839BFECF949A8C9810F094988C9A28
:1010C00093988B9A2FD08B98939A2CD08399F8CFA2
:1010D00018F0949A8C9802C094988C9A839BFECFB7
:1010E0008C98949A111F9A9521F7089501B3077D62
:1010F00001BB02B3086102BB99E08399FECF8894DB
:10110000849B06C0089493988B9A8499FECF04C060
:1011100093988B9A849BFECF8B98939A111F9A95E4
:1011200061F7089530E540E54A95F1F73A95D9F72A
:1011300008955F9B09C00CB1033111F4B06404C081
:0A1140000CB1033009F4B260089509
:00000001FF
